:020000040000FA
:02000000512984
:080008008E00030E8D00803014
:100010008107402046205A208F0A8F08031D382868
:10002000900A151C17289603031D17281510171C76
:100030001E28061F1D2806131E2806173C30100216
:10004000031D382890016E20171006131C08180293
:10005000031D38281D081902031D38281E081A021E
:10006000031D38281F081B02031D38280617171404
:10007000BA200B113B280D0E83008E0E0E0E0900C8
:10008000861B0800151404309600080013184E282B
:100090000618080013143230940008009403031D5E
:1000A0000800131015185628A0200800AD200430B1
:1000B00096000800111862288618080011143230C2
:1000C000920008009203031D0800111015186A28F9
:1000D0007A2008008D200430960008009F0A0A301C
:1000E0001F02031D08009F019E0A06301E02031D09
:1000F00008009E0103301D02031D852802301C02EA
:10010000031D85289D019C0108009D0A0A301D02DF
:10011000031D08009D019C0A080003301902031DFD
:10012000982802301802031D9828990198010800A8
:10013000990A0A301902031D08009901980A08005B
:100140009F0A0A301F02031D08009F019E0A063005
:100150001E02031D08009E0108009B0A0A301B02B4
:10016000031D08009B019A0A06301A02031D0800AD
:100170009A0108001518C5281C08A0001D08A10038
:100180001E08A2001F08A300CE281808A000190806
:10019000A1001A08A2001B08A300CE288C03031D8F
:1001A000D32804308C0001300C02031DDC280E30F3
:1001B00085002008A400F72802300C02031DE52862
:1001C0000D3085002108A400F72803300C02031D20
:1001D000EE280B3085002208A400F72804300C021A
:1001E000031DF728073085002308A400F7280030F6
:1001F0002402031D0029061186110612861208002A
:1002000001302402031D09290615861106128612E3
:10021000080002302402031D122906118615061259
:100220008612080003302402031D1B2906158615BB
:1002300006128612080004302402031D2429061128
:10024000861106168612080005302402031D2D298A
:100250000615861106168612080006302402031DB4
:100260003629061186150616861208000730240264
:10027000031D3F290615861506168612080008304C
:100280002402031D4829061186110612861608004D
:1002900009302402031D0800061586110612861671
:1002A00008008312850186018316283081001030F2
:1002B0008500833086008312A0308B008501810188
:1002C0000C3084008001840A50300402031D62292E
:1002D00004308C00323094009200043096000613F3
:0402E00071297129E6
:02400E00F23F7F
:104200002800430029004600610062007200690036
:10421000630065002000530069006E0063006500C4
:10422000720065002000320031002F0030003200A3
:0A4230002F0032003000300037008C
:00000001FF
